:040000000203CA32FB
:03000B00020026CA
:0100130032BA
:01001B0032B2
:0D00230002019DC0E0C0D0D53E1B753E041B
:10003000D52A17752A0AD52B11752B282008037588
:100040002B28D206B20880022130300031053274EC
:100050000AB5322A753200E52E2401D4F52E501E41
:10006000752E00E52D2401D4F52D7460B52D0F7586
:100070002D00E52C2401D4F52C5003752C00300103
:10008000310533740AB5332A753300E5312401D4C0
:10009000F531501E753100E5302401D4F53074601F
:1000A000B5300F753000E52F2401D4F52F500375BE
:1000B0002F0030043F200D3CD5323975320AE52E31
:1000C0002499D4F52E7499B52E19752E99E52D2401
:1000D00099D4F52D7499B52D1B752D59E52C2499BE
:1000E000D4F52CE52C452D452E7009C204752B64E2
:1000F000C206D20CD53F38753F0AD5363275366404
:10010000E5372401D4F5377460B53723753700E53A
:10011000382401D4F5387460B53814753800E539E1
:100120002401D4F53974A07424B53903753900005D
:10013000300D1485372E85382D85392C853731853E
:10014000383085392F800C300409852E31852D30CB
:10015000852C2F85902220043F200D3C20021B205F
:10016000130C200009D200752B32C206D20C3000CD
:1001700009201506C200D202D20A20031B20140C4B
:10018000200109D201752B32C206D20C30010920A0
:100190001606C201D203D20BD0D0D0E032C0E0C0EC
:1001A000D0C000209904C2986118E540B401024112
:1001B00002B40202414FB40302419C75400080002A
:1001C000200A0A200B0C201A1EC2996118754001E2
:1001D0008003754002754101758DF37598407587F0
:1001E000C0C2B474026114754101754003A2189233
:1001F00019758DF37598C07587C0D29BD2B4740100
:1002000061140541E541B4020474316114B403047E
:10021000E52C610FB40404E52C6110B40504E52D50
:10022000610FB40604E52D6110B40704E52E610FDB
:10023000B40804E52E6110B40904E5326110B40A73
:100240000474036114C20A7541007540006116050B
:1002500041E541B4020474326114B40304E52F6132
:100260000FB40404E52F6110B40504E530610FB448
:100270000604E5306110B40704E531610FB40804E9
:10028000E5316110B40904E5336110B40A04740364
:100290006114C20B75410075400061160541E541CE
:1002A000C29BB40210E54D54F06004E54D6114E5C5
:1002B0004D44F06114B40304E54E6114B4040CE53C
:1002C0004F300405200D0244FF6114B40510E550C1
:1002D00054F06004E5506114E55044F06114B40634
:1002E00004E5516114B4070CE552300405200D02F9
:1002F00074FF6114B40804E5436114B40904E544CF
:10030000611420191DC21A7541007540006116C4A0
:10031000540F2430F599C299754204D000D0D0D042
:10032000E032B40A0F758DF37598407587C0C2B47A
:1003300074026114B40B0E74333004077435300D3D
:100340000274366114B40C04E54D610FB40D04E57C
:100350004D6110B40E04E54E610FB40F04E54E611B
:1003600010B41004E54F610FB41104E54F6110B4EF
:100370001209E55330040274006110043004028055
:100380003FB4140474346114B41504E550610FB41F
:100390001604E5506110B41704E551610FB4180458
:1003A000E5516110B41904E552610FB41A04E55225
:1003B0006110B41B04E5546110B41C04740361148F
:1003C000C21A754100754000611675B0FF7590FF47
:1003D0007580FF75A0FF75816F758922758DE67533
:1003E0008C06752A28752BC8C206D2A9D28CD28E4B
:1003F000C2A8C2AAC29C7598C07587C0C298D2AC68
:10040000D2B9752000752100752200752300754151
:10041000007540007534037539087538007537006C
:10042000753F0A75366475435A754414D218D2AFB5
:1004300012097A1207CB752B64C2063006FD7900CB
:10044000120832752B1EC2063006FD7900120839DB
:10045000752B1EC2063006FD7900120840752B1E52
:10046000C2063006FD7900120847752B1EC2063001
:1004700006FD790012084F752B1EC2063006FD7965
:1004800000120857752B1EC2063006FD79001208AF
:100490005F752B14C2063006FD1209EB79071208AE
:1004A0001D794712081DD204C1C1E520540F600216
:1004B000A17B20043A209037753AFF753B04C20FA8
:1004C000C20E85342C75320A752D00752E00752FDD
:1004D00000753000753100C21DC21ED204D2071251
:1004E00009EB7900120801754410790712082B20D6
:1004F0000E2230900AD53A07D20FD53B02D20E20F9
:100500009012300F0FD20D790712082479001208CB
:100510000F754416E52C30044F30094C209116C25B
:1005200009200D1D2401D4F52CF534703B753401E0
:10053000752C018033209230C209200D1624998039
:10054000E5309021E5392401D4F539B4241A753900
:1005500000801530900FE5382401D4F538B46008D8
:10056000753800800375370020091030920A3091E9
:1005700007D53507D209800375353CA207B0045072
:1005800011C207790712081D794712081D75441416
:10059000C1C1A204B00D4009790D7C02784712094F
:1005A000FD790A7C0278461209FD79077C027845BC
:1005B0001209FD200407790F784B1209F520042554
:1005C000794D7C02784A1209FD794A7C02784912F9
:1005D00009FD79477C0278481209FD200407794F0C
:1005E000784C1209F57900301D083008051208080A
:1005F0008034790020046D300014309302D21B2027
:100600009303201B04F1EC801D12081680183002A1
:100610000C301B053093F2C21BF1F3800920A104BA
:10062000F1E58002F1FA7940301E08300805120821
:100630000880317940300114309402D21C20940398
:10064000201C04F1EC801D120816801830030C30B9
:100650001C053094F2C21CF1F3800920A004F1E5DE
:100660008002F1FA200416A2007202B3B097500281
:10067000D21DA2017203B3B0B25002D21E20B01E2E
:1006800020043E309667C201C203753300752F0007
:10069000753000753100C21CC21EC20FC20E20B3DD
:1006A0004C20041D309546C200C202753200752CE4
:1006B00000752D00752E00C21BC21DC20FC20E8018
:1006C0002CC2AFC204C20DD2AF75320075330075B3
:1006D0002F00753000753100752C00752D00752EBA
:1006E00000C21BC21CC21DC21EC20FC20EA200B39A
:1006F00092A4A201B392A3A20CB392A2300602C2AA
:100700000C200414209502C2A120B302D2A120968D
:1007100002C2A020B002D2A000A21DB008B392B5C0
:1007200000A21EB008B392B6E5407007D54204D2CD
:100730001AD29920043F200D3C30902D3091053085
:100740009216803130062EE54304C394645026058A
:1007500043752B0AC206801D30061AE54314601546
:100760001543752B0AC206800C209104D21880050F
:10077000209202C218200406301B03309310C2AF2F
:10078000852C45852D46852E4785324BD2AF0020DE
:100790000406301C03309410C2AF852F48853049C1
:1007A00085314A85334CD2AFC2AF852C4D852D4E55
:1007B000852E4F853253D2AF00C2AF852F50853082
:1007C00051853152853354D2AF81AA9008671209FE
:1007D000F07C5078008005120A247800E893120912
:1007E000A508DCF8229009517C0680EB9009277C53
:1007F0000680E490092E7C0680DD9009357C068019
:10080000D690093C7C0680CF9009437C0680C89036
:10081000094A7C0680C19009587C0680BA90095F1D
:100820007C0980B39009687C0980AC9009717C09CF
:1008300080A59008B77C10809E9008C77C10809798
:100840009008D77C1080909008E77C100207D79022
:1008500008F77C100207D79009077C100207D79091
:1008600009177C100207D73E2020202020202020BE
:100870002020202020203C2E2E2E2E2E2E2E2E2EDE
:100880002E2E2E2E2E2E2E2E2E2E2E2E2E2E2E486E
:1008900061736963692020446F6C2E447675722EF3
:1008A0002E2E2E2E2E2E2E2E2E2E2E2E2E2E2E2E68
:1008B0002E2E2E2E2E2E2E203E20202020202020B8
:1008C00020202020203C2020203E202020202020EE
:1008D000202020203C20202020203E2020202020DE
:1008E0002020203C202020202020203E20202020CE
:1008F00020203C2020202020202020203E202020BE
:10090000203C20202020202020202020203E2020AD
:100910003C202020202020202020202020203E3C81
:100920002020202020202053544152542020535472
:100930004F5020202052454144592020414C4152E3
:100940004D202020202020202020434C4F434B20AE
:10095000204552524F522020494E464F2020202001
:10096000203A20202E20202020203A20203A20202B
:100970002020203A2020202020207F327EFADEFE18
:10098000DFFA74301209B37F32DFFE74301209BA15
:1009900074381209BA740C1209BA74011209BA74C3
:1009A000061209BA22D2A5C2A6D38013D2A5C2A626
:1009B000C3800CC2A6C2A5C38005C2A6C2A5D3F53A
:1009C00080D2A7C2A7400822C3D2A5D2A6800CD34A
:1009D000C2A5D2A68005C3C2A5D2A67580FFD2A7A4
:1009E000E580C2A75004A2E740F12274011209BABF
:1009F00074800209BA7C01D2D580067C01C2D58000
:100A000000120A24120A0ADCFB22E620D501C45493
:100A10000F240630E40274F6242AB2D520D501084A
:0A0A2000090209A5E944800209BAA1
